:100000000C9434000C9451000C9451000C94510049
:100010000C9451000C9416010C9451000C94510056
:100020000C9451000C9451000C9451000C9451000C
:100030000C9451000C9451000C9451000C945100FC
:100040000C9482010C9451000C9451000C945100BA
:100050000C9451000C9451000C9451000C945100DC
:100060000C9451000C94510011241FBECFEFD8E026
:10007000DEBFCDBF11E0A0E0B1E0E4E3F4E002C0F8
:1000800005900D92A832B107D9F721E0A8E2B1E0BE
:1000900001C01D92A733B207E1F70E94F9010C9449
:1000A00018020C940000E1ECF0E0108286E08093EE
:1000B000C20083E390E09093C5008093C4008081E8
:1000C000886180838091C60008959091C00095FF5B
:1000D000FCCF8093C6000895CF93DF93EC0102C05C
:1000E0000E94650089918111FBCF8DE00E9465001F
:1000F0008AE0DF91CF910C9465006F927F928F928E
:100100009F92AF92BF92CF92DF92EF92FF920F93A6
:100110001F93CF93DF93CDB7DEB7A8970FB6F894B0
:10012000DEBF0FBECDBF38E2E0E0F1E0DE011196A8
:1001300001900D923A95E1F7AAE0AA2EA21A97FF34
:100140000BC090958095709561957F4F8F4F9F4F15
:100150002DE2FA012193AF01DE01119620E030E09B
:10016000EA2DFF27E7FDF0953197B22E2E173F07B6
:1001700064F4CD90DD90ED90FD902F5F3F4F6C15B6
:100180007D058E059F0588F32B2DDE011196F4E089
:100190002F02A00DB11D1124612C712CFEE28F2EB7
:1001A00001C0A701BA1003C0FA018192AF019D01FD
:1001B000260D371DF9010081118122813381E0E391
:1001C0009E2ECC24DD247601C01AD10AE20AF30A5D
:1001D00005C093946C0D7D1D8E1D9F1D60177107CA
:1001E00082079307B0F7B394FA0191927F01F4E08C
:1001F0006F0E711C013011052105310591F6FA01D0
:100200001182A8960FB6F894DEBF0FBECDBFDF9166
:10021000CF911F910F91FF90EF90DF90CF90BF9003
:10022000AF909F908F907F906F9008951F920F9244
:100230000FB60F9211242F938F939F9389B18C70D7
:100240009BB1982B9BB99AB19C609AB99091280167
:1002500098278093280192FF07C0811102C021E0F6
:1002600008C08C30E1F304C08430C9F38830B9F39E
:100270002FEF80912E0190912F01820F911D27FD6C
:100280009A9590932F0180932E018AB1837F8AB92A
:100290008BB1837F8BB984E08BBB9F918F912F9122
:1002A0000F900FBE0F901F9018950F931F938FB74D
:1002B000F89400912A0110912B0120912C0130918A
:1002C0002D018FBFB801C9011F910F910895EDE66F
:1002D000F0E080818460808380818860808384E016
:1002E0008BBBE8E6F0E08081846080837894089599
:1002F00085E085BD81E085BBEEE6F0E08081816030
:10030000808308951F920F920FB60F9211242F939E
:100310003F934F935F936F937F938F939F93AF938D
:10032000BF93809129018F5F80932901853008F464
:1003300051C080916E008E7F80936E0010922901D3
:1003400040912E0150912F0110922F0110922E01F9
:10035000789457FF02C04F5F5F4F55954795CA018C
:1003600057FF04C088279927841B950B833091057C
:10037000A4F0459714F4CA0102C084E190E0889F7C
:100380009001899F300D300D112457FF05C044277F
:100390005527421B530B01C0A90180912A0190915E
:1003A0002B01A0912C01B0912D01662757FD60957E
:1003B000762F841B950BA60BB70B80932A01909385
:1003C0002B01A0932C01B0932D0180916E008160D0
:1003D00080936E00BF91AF919F918F917F916F91AC
:1003E0005F914F913F912F910F900FBE0F901F90F3
:1003F00018950E9467010E9478010E945300812C89
:10040000912C54010E9455016B017C0168157905FE
:100410008A059B05B9F322E040E351E0C7010E9441
:100420007D0080E391E00E946C0046015701EACF15
:04043000F894FFCF6E
:1004340000CA9A3B00E1F5058096980040420F00FF
:10044400A086010010270000E803000064000000FB
:080454000A0000000100000095
:00000001FF
